:0300000002457145
:0C45710078FFE4F6D8FD7581610245B8C2
:101E150020000A3C2E2E2E3E004950436F6E6E6503
:101E250063745245510A004950436F6E6E65637481
:101E3500000A49504E6F41434B210A003E432C5640
:101E45002C43432CC0E4E0EFF2E5F020D1E8EDEAC5
:101E5500EEEC49500A003E432C4D41432C253032CF
:101E650062583A25303262583A25303262583A255E
:101E7500303262583A25303262583A25303262584B
:101E85002C4D414320E0E4F0E5F10A003E432C5699
:101E950045522C20332E3220EEF220257320257357
:101EA5002CC2E5F0F1E8FF20495020ECEEE4F3EB1D
:101EB500FF0A00417072203138203230303800314D
:101EC500303A35373A3135003E432C4C442C50528C
:101ED5004F473A202020202020202020202020208D
:101EE50020202020202020202020202020202020ED
:101EF50020202020202020202020202020202020DD
:101F050020202020202020202020202020202020CC
:101F150020202020202020202CC4E0F2E020EFF01B
:101F2500EEF8E8E2EAE828F4E0E9EB290A003E2ABF
:101F35002C312CCEF1EDEEE2EDFBE520EFE0F0E00B
:101F4500ECE5F2F0FB20F1E5F2E5E2EEE3EE20E868
:101F5500EDF2E5F0F4E5E9F1E00A003E412C41300F
:101F6500312C2562752E2562752E2562752E25620A
:101F7500752C495020E0E4F0E5F120E0E4E0EFF2D3
:101F8500E5F0E00A003E412C4130322C2562752EE9
:101F95002562752E2562752E2562752C495020E027
:101FA500E4F0E5F120EEF1ED2E20F1E5F0E2E5F0CB
:101FB500E00A003E412C4130332C2562752E256206
:101FC500752E2562752E2562752C495020E0E4F0AA
:101FD500E5F120F0E5E72E20F1E5F0E2E5F0E00A95
:101FE500003E412C4130342C2562752E2562752E1C
:101FF5002562752E2562752CCCE0F1EAE020F1E52D
:10200500F2E80A003E412C4130352C2562752E251B
:1020150062752E2562752E2562752CD8EBFEE70AB2
:10202500003E2A2C312CC4EEEF2E20EFE0F0E0EC40
:10203500E5F2F0FB20F1E5F2E5E2EEE3EE20E8ED76
:10204500F2E5F0F4E5E9F1E00A003E422C533031C7
:102055002C2562752CC6E4E0F2FC20E7E0EFF0EEFB
:10206500F1E020F1EEE5E4E8EDE5EDE8FF20EEF244
:1020750020F1E5F0E2E5F0E00A003E422C53303273
:102085002C2562752CCEE1ECE5ED20F120F1E5F093
:10209500E2E5F0EEEC20E1E5E720EAE2E8F2E0ED4A
:1020A500F6E8E90A003E422C5330332C2562752CA4
:1020B500CFE5F0E5E7E0EFF3F1EA20EFF0E820EF18
:1020C500EEF2E5F0E520F1E2FFE7E820F120F1E5A9
:1020D500F0E2E5F0EEEC0A003E422C5330352C25BB
:1020E50062752CCAE0EDE0EB20F8E8F0EEEAEEE2EE
:1020F500E5F8E0F2E5EBFCEDEEE3EE20EEE1ECE5F4
:10210500EDE00A003E532C5330362C253032625810
:1021150025303262582530326258253032625825D2
:102125003032625825303262582C4D414320E0E46C
:10213500F0E5F120F8E8F0EEEAEEE2E5F8E0F2E5A8
:10214500EBFCEDEEE3EE20EEE1ECE5EDE00A003E22
:10215500454E440A000A44756D7058202020202001
:1021650030302030312030322030332030342030B0
:102175003520303620303720303820303920304176
:102185002030422030432030442030452030460066
:102195000A3A003A20000A000A44756D704420206E
:1021A5002020203030203031203032203033203094
:1021B5003420303520303620303720303820303943
:1021C500203041203042203043203044203045200B
:1021D500304600457272206B657900526420656552
:1021E50070726F6D0A005264204D454D0A005264AD
:1021F50020436F64650A00577269746520436F64F4
:10220500650A0044656275674950204F4E0A0044CF
:10221500656275674950204F46460A0044656275F8
:102225006755736572204F6E0A0044656275675580
:10223500736572204F46460A0044656275674D73A3
:1022450067204F6E0A0044656275674D7367204FBE
:1022550046460A00436F6E666967206C6F636B21A3
:102265000A00577220656570726F6D0A0020536110
:10227500766520656570726F6D210A004572722062
:102285004D414321004C6F61643E3E002A003C41B4
:1022950030313D003C4130323D003C4130333D0062
:1022A5003C4130343D003C4130353D003C21003C53
:1022B5005330313D003C5330323D003C5330333DCB
:0D22C500003C5330353D003C5330363D00A9
:06503F00015E00015C00AF
:10500200C28E438910758BFF758DB7D2ABD28E22BB
:03001B000244E1BB
:1044E100C0E0C083C082C0D0C28E758BFF758DB70E
:1044F10020060675A61E75A6E1055CD202E55E6082
:1045010002055EE55DD394014002155D0561E5613B
:10451100540F7048D20EE561543F7012D200906E74
:10452100C5E0600A04F0E0D394B44002D206906E74
:10453100C0E0600204F090693EE0600214F0906E09
:10454100C6E0D394014003E014F0300502055FE5B5
:1045510060D394644004D20680020560E55BD39485
:10456100014002155BD28ED0D0D082D083D0E03210
:1017B300C2AFC291C290D2B5C20B7D027C007F073B
:1017C300124FA38F26E526646060097D017F6012B6
:1017D3004F3ED20BE4FDFC7F0B124FA38F26E52671
:1017E30030E6097D04E4FF124F62D20B7D017C00D9
:1017F3007F07124FA38F26E5267008FD7FFF124F48
:101803003ED20B300B03126000C288C2A8C2AA7575
:1018130089001249A9906B78E0B4FA06A3E064CE7C
:10182300607BE4F52674702526F582E4346BF5833A
:10183300E4F00526E526B443EC906B7874FAF0A344
:1018430074CEF0A374CCF0906B7E740AF0E4A3F032
:10185300A304F0A3F0906B7474FFF0A3F0A3F0E47F
:10186300A3F0906B8F740AF0E4F526E5262401FFBC
:10187300E433FE74702526F582E4346BF583E0FDD2
:10188300124F1A0526E526C3944340DFE4F5A775F6
:10189300A61E75A6E1907FF0F0A3F080FE906B8307
:1018A3007403F0A374CCF0E4906B82F012415BC23A
:1018B300B5123293C206124C9ED20BC20DC20C90CB
:1018C3006DB07408F0906AEE7424F0E4A3F0906BAA
:1018D30078E0906AF0F0906B79E0906AF1F0906BA9
:1018E3007AE0906AF2F0906B7BE0906AF3F0906B91
:1018F3007CE0906AF4F0906B7DE0906AF5F0755DA2
:1019030001E4906DB1F0C207C208C209C20A124EC7
:10191300F3200B19AF267E007D03123F9FE4FF12D5
:10192300439A7E1E7F15E4FBFDFC123CAC906EC512
:10193300E060037401F0E490693EF0F55F906DAFF1
:10194300F0F56012500275A70775A61E75A6E1D2C1
:10195300AFE4F56090693EE0700312262E906EC6E8
:10196300E0B401119080007410F0E4906EC6F0D2E0
:101973000BC20CC20D908008E0F52630E405D207B7
:101983007410F0E52630E508D2099080087420F041
:10199300E52630E608D2089080087440F0E55FC37E
:1019A30094034019908002E4F0908001F09080004D
:1019B300F0E55F94064006E4F55F124C9E9080A02C
:1019C300E07003124A279080B8E07003124AA19096
:1019D30080D0E07003124B1B908000E0701330073F
:1019E30010123DB3906B6BEFF0D3940040031208D9
:1019F300E2908002E07006908000E06005D205026C
:101A03001954C205E4F55F90693EE060030219547E
:101A1300200B12906DB2E0600C7E1E7F17123EB752
:101A2300E4906DB2F03009121238D5906B6BEFF081
:101A3300D394004005E0FF125012200803021BBD9F
:101A43001235DF906B6BEFF07003021954906BAF9C
:101A5300E054BF247F7003021B26147003021AFE96
:101A630024026003021B5F200B077E1E7F1E123EB3
:101A7300B7200F03021BBD906B87E07006906B8B42
:101A8300E06067906EBCE0FF906B87E0B507249041
:101A93006EBDE0FE906B88E0B50618906EBEE0FE6A
:101AA300906B89E0B5060C906EBFE0FE906B8AE008
:101AB3006E6037906B8BE06F6003021BBD906EBD51
:101AC300E0FF906B8CE06F6003021BBD906EBEE085
:101AD300FF906B8DE06F6003021BBD906EBFE0FF54
:101AE300906B8EE06F6003021BBDC203906DB174F7
:101AF30001F0120021755D01021BBD906EC5E0600F
:101B0300037401F0906EB4E0FF906BB1E06F60037B
:101B1300021BBD906EB4E004F0E4F55D906DAFF090
:101B2300021BBD300303021BBD906B7EE0700302FA
:101B33001954906B8F740AF0125046D203E4F55D8A
:101B4300906DAFF0906EC004F0E4906EB3F0A3F02C
:101B5300200B677E1E7F2C123EB7805E906EC5E021
:101B630060037401F0300352906BAFE020E74B90B9
:101B73006BB1E0FF906EB3E0FE6F600D906EBBE063
:101B83007007EE146F70338013906EB3E004F0901F
:101B93006B6BE0FFD394044003124D8590683A7455
:101BA30082F0A37401F0906BB1E090683CF07E6822
:101BB3007F3A7D03124710021954200303021CD5F8
:101BC300E55D7068124E6AEF60237E6C7FAF906CA8
:101BD300B0E02404FD124710906EBBE07009906BD7
:101BE3008FE0F55D021954E4F55D021954906EC05F
:101BF300E0D3943C4036906EBBE07030906EC004EE
:101C0300F012502CE4906CAFF0A37412F0906EB409
:101C1300E0906CB1F0A374FDF090693F63A2019072
:101C23006CB363A2017F12123185809E1250218F03
:101C330026E526B4011590683A7483F0E4A3F07E98
:101C4300687F3A7D02124710021954E526D39401A6
:101C5300401C90683A7483F0A37401F0E52624FED7
:101C6300A3F07E687F3A7D03124710021954E55DA5
:101C730064016003021954906DAFE004F0200B0778
:101C83007E1E7F36123EB7906B8FE0C394C850041C
:101C9300E02432F0906DAFE0C39405400DC203E43D
:101CA300906DB1F01200210219547C6E7DBC906BD3
:101CB30083E0FAA3E0FB7F021248A17E6C7FAF9022
:101CC3006CB0E02404FD124710906B8FE0F55D02C9
:101CD3001954E55D64016003021954906DB1E01479
:101CE300604624FE6042147003021DC8240460038E
:101CF300021954E4F55F200F13906DB17404F09052
:101D03006DAFE05401F0755D0102195490800274C7
:101D130010F0E4906DB1F0906DAF04F0755DFA9042
:101D23006EBC74FFF0021954906EBCE07003021D88
:101D3300B2906CAF7480F0906CB17401F0E4A3F0D6
:101D4300A304F0A37430F0A3747BF0E4F52674B617
:101D53002526F582E4346CF583747DF074B725266B
:101D6300F582E4346CF583E4F0E5262407906CB047
:101D7300F07C6E7DBC906B83E0FAA3E0FB7F0212E4
:101D830048A17E6C7FAFE5262409FD124710906EB3
:101D9300BBE0601B125046D203E4F55D906DAFF0DB
:101DA300906EC004F0E4906EB3F0A3F002195430C7
:101DB3000F07E4906DB1F08006906DB17404F07577
:101DC3005DFA0219549080027410F0755D05906DF0
:101DD300AFE06401FFF0906DB17401F0EF70199002
:101DE3006B8BE06013FCA3E0FDA3E0FEA3E0FF9098
:101DF3006EBC122AC0021954906B87E0FCA3E0FD6D
:101E0300A3E0FEA3E0FF906EBC122AC00219548027
:011E1300FED0
:011E140022AB
:1008E200906BB0E0B444047F0180027F00906BAF54
:1008F200E0B447047E0180027E00EE5F604A906BA6
:1009020078E0906BB1F0906B79E0906BB2F0906B05
:100912007AE0906BB3F0906B7BE0906BB4F0906BED
:100922007CE0906BB5F0906B7DE0906BB6F0906BD5
:10093200B07452F0906AE863A2019080A863A201A9
:100942007F06123185021137906B6BE0C394085019
:1009520003021140906B78E0FF906BB1E06F60038F
:10096200021140906B79E0FF906BB2E06F6003027E
:100972001140906B7AE0FF906BB3E06F600302115D
:1009820040906B7BE0FF906BB4E06F60030211401C
:10099200906B7CE0FF906BB5E06F600302114090BA
:1009A2006B7DE0FF906BB6E06F6003021140906BCD
:1009B200B0E0B44415906AE8E0B4FF0E63A201907F
:1009C20080A863A2017F06123185906EC5E06003A4
:1009D2007401F0906EC67464F0906BB07452F09033
:1009E2006BAFE0646D6003020B417BFF7A1E7941BD
:1009F2001223347BFF7A1E795B906B78E0F52FA38C
:100A0200E0F530A3E0F531A3E0F532A3E0F533A33E
:100A1200E0F534122334752FFF75301E7531B87529
:100A220032FF75331E7534C47BFF7A1E799112230F
:100A3200347BFF7A1E79CD1223347BFF7A1F793300
:100A42001223347BFF7A1F7960906B7EE0F52FA32F
:100A5200E0F530A3E0F531A3E0F5321223347BFF59
:100A62007A1F798A906B87E0F52FA3E0F530A3E037
:100A7200F531A3E0F5321223347BFF7A1F79B89067
:100A82006B8BE0F52FA3E0F530A3E0F531A3E0F5A1
:100A9200321223347BFF7A1F79E6906B74E0F52FD4
:100AA200A3E0F530A3E0F531A3E0F5321223347B65
:100AB200FF7A207909906B70E0F52FA3E0F530A35F
:100AC200E0F531A3E0F5321223347BFF7A20792658
:100AD2001223347BFF7A20794FA20FE433F52F12D1
:100AE20023347BFF7A20797F906EBBE0F52F1223AF
:100AF200347BFF7A2079AA906EC5E0F52F12233459
:100B02007BFF7A2079DDA201E433F52F1223347BB7
:100B1200FF7A217909906EB5E0F52FA3E0F530A3B5
:100B2200E0F531A3E0F532A3E0F533A3E0F53412AA
:100B32002334123B937BFF7A21795412233422907F
:100B42006BAFE0644C70737E217F5AFBFDFC123C5C
:100B5200AC906BB7E0F527A3E0F528E4F52AE5278A
:100B6200906BB9F0A3E528F07E217F957C6B7DB96F
:100B72007B02123CACE4F529852882852783E0FFBD
:100B820074B92529F582E4346BF583EFF00528E585
:100B920028700205270529E529B410DC7E217F98FB
:100BA2007C6B7DB97B10123CAC052AE52AC39410FC
:100BB20040AC7E217F9B123EB722906BAFE0646C0B
:100BC2007060F52B7E217F9DFBFDFC123CACE4F5B1
:100BD2002AE4906BB9F0A3E52BF07E217F957C6B24
:100BE2007DB97B02123CACE4F529A82BE6FF74B96F
:100BF2002529F582E4346BF583EFF0052B0529E511
:100C020029B410E67E217F987C6B7DB97B10123C63
:100C1200AC052AE52AC3940840B77E217F9B123E89
:100C2200B722906BAFE0644B7061F52974A125295E
:100C3200F582E4346BF583E0603274A12529F582F4
:100C4200E4346BF583E0F4602374A12529F582E492
:100C5200346BF583E0FF74B72529F582E4346BF534
:100C620083E0B507100529E529B408C090693E74F0
:100C720032F0021137906BAF7421F0300B03021186
:100C8200377E217FD8123EB7021137906BAFE0B4A6
:100C9200521A200B077E217FE0123EB7906BAF7491
:100CA20072F07E6B7FAF7D0812468922906BAFE0B7
:100CB20064497045200B077E217FEB123EB7906B93
:100CC200B7E0F527A3E0F528E4F5298528828527F2
:100CD20083E0FF74B92529F582E4346BF583EFF0E4
:100CE2000528E528700205270529E529B480DC7E60
:100CF2006B7FAF7D8A12468922906BAFE0644370AE
:100D020046200B077E217FF3123EB7906BB7E0F5CA
:100D120027A3E0F528E4F529852882852783E49333
:100D2200FF74B92529F582E4346BF583EFF00528C9
:100D3200E528700205270529E529B480DB7E6B7F53
:100D4200AF7D8A12468922906BAFE0645A705320BD
:100D52000B077E217FFC123EB7906BB7E0F527A30D
:100D6200E0F5287C6B7DB97B80AF28AE27124E362A
:100D7200E4F529852882852783E493FF74B9252920
:100D8200F582E4346BF583EFF00528E5287002055F
:100D9200270529E529B480DB7E6B7FAF7D8A124669
:100DA2008922906BAFE064446003020E35906BB70A
:100DB200E0FF64447003021137EFB4310CC20B7EC2
:100DC200227F08123EB7021137906BB7E0B4300CA5
:100DD200D20B7E227F14123EB7021137906BB7E01E
:100DE200B4320CD20C7E227F21123EB70211379010
:100DF2006BB7E0B4330CC20C7E227F2F123EB702D7
:100E02001137906BB7E0B4340CD20D7E227F3E12C4
:100E12003EB7021137906BB7E0B4350CC20D7E229B
:100E22007F4B123EB7021137906BB7E0FF12001EE4
:100E320002113790693EE07013200B077E227F5922
:100E4200123EB7906BAF7421F002113790693E7475
:100E520032F0906BAFE0FFB45104C2AF80FEEF649A
:100E6200577045200B077E227F67123EB7906BB802
:100E7200E0906B6BF0E4F529906B6BE0FFE529C322
:100E82009F400302113774B92529F582E4346BF5CA
:100E920083E0FF906BB7E0252924E7F582E434690B
:100EA200F583EFF0052980D0906BAFE064536003C7
:100EB200020F58200B077E227F72123EB7906B788A
:100EC200E0FF9069F0E06F703C906B79E0FF906911
:100ED200F1E06F7030906B7AE0FF9069F2E0B50755
:100EE20024906B7BE0FF9069F3E0B50718906B7C70
:100EF200E0FF9069F4E0B5070C906B7DE0FF90692C
:100F0200F5E06F6016906BAF7421F0300B030211A5
:100F1200377E227F81123EB7021137E4F529E4F5CC
:100F220060AF29FE74E72529F582E43469F583E090
:100F3200FD124F1A0529E529C394FE40E1C2AFE430
:100F4200907FF0F0A3F0907FFD74AAF0A374FFF0FD
:100F5200A37455F080FE906BAFE0644F704C906BC1
:100F6200B7E0F527A3E0F528E5284527700A200B0E
:100F7200077E227F8A123EB7200B077E227F9112C4
:100F82003EB7E4F52974B92529F582E4346BF5837B
:100F9200E0852882852783F00528E5287002052749
:100FA2000529E529B480DE021137906BAFE0FFB46A
:100FB2004521906BB7E0FDA3E0907FF0CDF0A3ED6B
:100FC200F0C2AF907FFD74AAF0A374FFF0A3745532
:100FD200F080FEEF64656003021140906BB7E0FFA2
:100FE200A3E0907FF0CFF0A3EFF0E4F527F528D34C
:100FF200907FF1E09528907FF0E095274020E4F57E
:10100200602528FFE5273401FE852882852783E0B5
:10101200FD124F1A0528E5287002052780D17E228D
:101022007F93124797EF4E6020120003906B7EEF82
:10103200F0120003906B7FEFF0120003906B80EFD1
:10104200F0120003906B81EFF07E227F9912479796
:10105200EF4E6020120003906B87EFF012000390B6
:101062006B88EFF0120003906B89EFF0120003908F
:101072006B8AEFF07E227F9F124797EF4E6020121D
:101082000003906B8BEFF0120003906B8CEFF01269
:101092000003906B8DEFF0120003906B8EEFF07EE9
:1010A200227FA5124797EF4E6020120003906B74C7
:1010B200EFF0120003906B75EFF0120003906B7665
:1010C200EFF0120003906B77EFF07E227FAB1247B6
:1010D20097EF4E6020120003906B70EFF012000346
:1010E200906B71EFF0120003906B72EFF01200033D
:1010F200906B73EFF0E4F529E4F560E5292401FF34
:10110200E433FE74702529F582E4346BF583E0FD47
:10111200124F1A0529E529C3944340DCC2AFE4907B
:101122007FF0F0A3F0907FFD74AAF0A374FFF0A308
:0E1132007455F080FE7E6B7FAF7D08124689FB
:01114000228C
:104DFE00AE07EEC39430400BEED394395005EE243B
:104E0E00D0FF22EEC39461400BEED394665005EEB4
:104E1E0024A9FF22EEC39441400BEED394465005D5
:084E2E00EE24C9FF22AF0622A9
:104FC000906AE7E004F07006906AE6E004F0906A08
:0A4FD000E6E0FEA3E0FF124F862288
:10000300124FC0124DFEEFC454F0FEC006124FC093
:08001300124DFED0E02FFF2288
:104C4100E490701FF0124FC0907020EFF0C39430C9
:104C51004018E0FFD39439501190701FE0243FF5C4
:104C610082E43469F583EFF0801190701FE0243FF6
:104C7100F582E43469F583E4F0800C90701FE00460
:104C8100F0E0D3940840BE753200753300753400EE
:0C4C9100E4F5357B017A69793F12343B71
:014C9D0022F4
:044797008E2C8F2DA8
:10479B00906AE6E4F0A374FFF0124FC0EF606EF482
:1047AB00606B852D82852C83E493B507EC752E0108
:1047BB00E52D252EF582E4352CF583E493602590C9
:1047CB006AE7E0252EFF906AE6E03400FE124F8682
:1047DB00E52D252EF582E4352CF583E493B50704FE
:1047EB00052E80CCE52D252EF582E4352CF583E4C2
:1047FB009370A6E52E24FFFFE434FFFE906AE7E0FA
:10480B002FF0906AE6E03EF07E007F0122E4FEFF8F
:01481B00227A
:10415B007E227FB1124797EF4E70037F01227E22A2
:10416B007FB4124797EF4E600C124FC0EF24D02450
:10417B00FF920F8002D20F7E227FBA124797EF4E2B
:10418B00600C124FC0EF24D0906EBBF08005E49012
:10419B006EBBF07E227FC0124797EF4E600C124F22
:1041AB00C0EF24D0906EC5F08005E4906EC5F07E14
:1041BB00227FC6124797EF4E600C124FC0EF24D0F0
:1041CB0024FF92018002C201906B7863A201906E72
:1041DB00B563A2017F0612318530013B7E227FCC75
:1041EB00124797EF4E6030120003906EB5EFF0124E
:1041FB000003906EB6EFF0120003906EB7EFF01263
:10420B000003906EB8EFF0120003906EB9EFF0124E
:0A421B000003906EBAEFF07F00225E
:104CF700906DB0E0C3947C503D906DB0E0FE04F041
:104D070074EE2EF582E4346AF583EFF0BF0A27903C
:104D17006DB0E0FF04F074EE2FF582E4346AF5839A
:104D2700E4F0906DB0E0FF12481C906DB07408F08D
:074D3700906AEFE004F02296
:104C9E009080007480F0906B7063A201F583F582B2
:104CAE0063A2017F08123185906B7863A201908018
:104CBE008863A2017F0A123185908092E4F0A3747A
:104CCE0032F0A37401F0906B82E0FF9080B1F0900F
:104CDE0080E1EFF09080957455F0A3F09080007411
:094CEE0001F090800974F0F0223D
:104A2700908009E04410F09080A0E0706C9080A125
:104A37007482F09080A874FFF0A3F0A3F0A3F07F36
:104A4700039080AEEFF07FCBA3EFF07F039080ACB5
:104A5700EFF0A374CBF09080007402F09070131203
:104A67002ACC00000000907013E0908040F0907016
:104A770014E0908041F0907015E0908042F09070C3
:104A870016E0908043F0A3E4F0A3F0A3F0A3F09026
:094A97008018F0A3F0A3F0A3F0D5
:014AA00022F3
:104B1B00908009E04440F09080D17482F0906B83D8
:104B2B00E0FF9080DEF0906B84E0FF9080DFF090F0
:104B3B0080027402F0907017122ACC0000000090D3
:104B4B007017E0908058F0907018E0908059F090BA
:104B5B007019E090805AF090701AE090805BF0A38F
:104B6B00E4F0A3F0A3F0A3F0908030F0A3F0A3F057
:024B7B00A3F0A5
:014B7D002215
:104AA100908009E04420F09080B8E0706C9080B96B
:104AB1007482F07F039080C6EFF07FCDA3EFF07F8B
:104AC100039080C4EFF0A374CDF09080C074FFF028
:104AD100A3F0A3F0A3F09080017402F090701B1278
:104AE1002ACC0000000090701BE090804CF0907088
:104AF1001CE090804DF090701DE090804EF0907021
:104B01001EE090804FF0A3E4F0A3F0A3F0A3F09097
:094B11008024F0A3F0A3F0A3F04E
:014B1A002278
:1048A1008C278D28A907EAFDE975F018A424ACFF2F
:1048B100E5F034808F82F583EDF0EBFDE975F018BA
:1048C100A4FFAEF024ACFBEE34808B82F583A3ED24
:1048D100F08528828C83E0FDEF24A8FFEE3480FE72
:1048E1008F82F583EDF08528828C83A3E08F828E01
:1048F10083A3F0852882852783A3A3E0FDE975F0D2
:1049010018A424A8FFE5F03480FE8F82F583A3A3C9
:10491100EDF08528828C83A3A3A3E08F828E83A3ED
:04492100A3A3F0223A
:064689008D2CAB07AA0610
:10468F00908000E030E507906DB27401F0229070D9
:10469F0013E0FCA3E0FDA3E0FEA3E0F5308E2F8D29
:1046AF002E8C2DAE02AF038E838F8263A201E52F76
:1046BF00540744C0F58385308263A201AF2C1231B9
:1046CF00F7E4FCFDFEE530252CF530EE352FF52F08
:1046DF00ED352EF52EEC352DF52D908040E52DF096
:1046EF00A3E52EF0A3E52FF0A3E530F09080007442
:1046FF0020F0AF30AE2FAD2EAC2D907013122AC01C
:01470F002287
:064710008D27AB07AA068D
:10471600908002E030E507906DB27403F02290704D
:1047260017E0FCA3E0FDA3E0FEA3E0F52B8E2A8DA7
:10473600298C28AE02AF038E838F8263A201E52AFD
:10474600540744D0F583852B8263A201AF2712312B
:10475600F7E4FCFDFEE52B2527F52BEE352AF52A99
:10476600ED3529F529EC3528F528908058E528F00F
:10477600A3E529F0A3E52AF0A3E52BF090800274C7
:1047860020F0AF2BAE2AAD29AC28907017122AC0A4
:014796002200
:02439A008F286A
:10439C00908001E030E509906DB27402F07F00224C
:1043AC0090701BE0FCA3E0FDA3E0FEA3E0F52C8ED7
:1043BC002B8D2A8C29906EB563A201E52B540744F2
:1043CC00C8F583852C8263A2017F0612320DE52C81
:1043DC002406F52CE4352BF52BE4352AF52AE435A7
:1043EC0029F529906DB363A201E52B540744C8F558
:1043FC0083852C8263A201AF2812320DE4FCFDFEF2
:10440C00E52C2528F52CEE352BF52BED352AF52A48
:10441C00EC3529F52990804CE529F0A3E52AF0A389
:10442C00E52BF0A3E52CF09080017420F0AF2CAEBE
:0D443C002BAD2AAC2990701B122AC0AF28AE
:014449002250
:103DB3009081E0E0F5270527052705270527052737
:103DC30005270527052705270527908010E0F52AF5
:103DD300A3E0F52BA3E0F52CA3E0F52D9081E1E022
:103DE300F527052705270527052705270527052780
:103DF300052705270527908014E0F52EA3E0F52F6E
:103E0300A3E0F530A3E0F531E530B52C08E531B595
:103E13002D037F0022E4F527E530540744E0F583C2
:103E230085318263A201906BAF63A2017F081232D6
:103E33003D906BB163A201906AE863A2017F061211
:103E43003185906BAFE0F528A3E0F529E4F52790E1
:103E53006BAFE0702AA3E024F8F527E5305407445C
:103E6300E0F58385318274082582F582E43583F594
:103E73008363A201906BAF63A201AF2712323DAE01
:103E830028E4FCFDE5312529F531E5303EF530ED3B
:103E9300352FF52FEC352EF52E908014E52EF0A35B
:103EA300E52FF0A3E530F0A3E531F09080007440F6
:033EB300F0AF2746
:013EB60022E9
:1035DF009081E6E0F527052705270527052705270D
:1035EF0005270527052705270527908028E0F52AB9
:1035FF00A3E0F52BA3E0F52CA3E0F52D9081E7E0F8
:10360F00F52705270527052705270527052705275B
:10361F0005270527052790802CE0F52EA3E0F52F31
:10362F00A3E0F530A3E0F531E4F527E530B52C0A3A
:10363F00E531B52D05C20802374BE530540744F08C
:10364F00F58385318263A201906BAF63A2017F087E
:10365F0012323D906BAFE0F528A3E0F529E529453F
:10366F002870099080027410F07F0022906EBCE0E9
:10367F00FFF46030906BB1E06F6003023712906E11
:10368F00BDE0FF906BB2E06F7079906EBEE0FF907F
:10369F006BB3E06F706D906EBFE0FF906BB4E06F37
:1036AF006031805F906BB1E0906EBCF0906BB2E0D8
:1036BF00906EBDF0906BB3E0906EBEF0906BB4E087
:1036CF00906EBFF0906BB5E0FFA3E0906B83CFF0EF
:1036DF00A3EFF0906BAFE0702AA3E024F8F527E595
:1036EF0030540744F0F58385318274082582F582C2
:1036FF00E43583F58363A201906BAF63A201AF271B
:10370F0012323DAE28E4FCFDE5312529F531E530D7
:10371F003EF530ED352FF52FEC352EF52EAF2DAEC6
:10372F002CAD2BAC2AAB31AA30A92FA82ED3122A3D
:10373F00AF40099080027410F07F002290802CE53A
:10374F002EF0A3E52FF0A3E530F0A3E531F0908044
:06375F00027440F0AF27E8
:013765002241
:1038D5009081E3E0F5270527052705270527052717
:1038E5000527052705270527052790801CE0F52ACC
:1038F500A3E0F52BA3E0F52CA3E0F52D9081E4E002
:10390500F527052705270527052705270527052762
:10391500052705270527908020E0F52EA3E0F52F44
:10392500A3E0F530A3E0F531E4F527E530B52C0A41
:10393500E531B52D05C209023A20E530540744E8C2
:10394500F58385318263A20190683E63A2017F0EF3
:1039550012325390683EE0F528A3E0F529906846B9
:10396500E0FFF46045906EB5E0FEEF6E706EA3E08B
:10397500FF906847E06F7064906EB7E0FF9068480D
:10398500E06F7058906EB8E0FF906849E06F704C3A
:10399500906EB9E0FF90684AE06F7040906EBAE0B3
:1039A500FF90684BE06F60048032D2D990683EE0AA
:1039B500702AA3E024F2F527E530540744E8F5839F
:1039C500853182740E2582F582E43583F58363A201
:1039D5000190683E63A201AF27123253AE28E4FC82
:1039E500FDE5312529F531E5303EF530ED352FF58D
:1039F5002FEC352EF52EAF2DAE2CAD2BAC2AAB31E1
:103A0500AA30A92FA82ED3122AAF5006E52945289A
:103A150070099080017410F07F0022908020E52EBF
:103A2500F0A3E52FF0A3E530F0A3E531F090800198
:053A35007440F0AF2712
:013A3A002269
:043EB7008E2D8F2E8F
:103EBB00908000E030E507906DB27401F0229070B5
:103ECB0013E0FCA3E0FDA3E0FEA3E0F5348E338DFD
:103EDB00328C31E534FFE5335407FEE42FF530EE39
:103EEB0034C0F52F853082F5837423F00530E5302F
:103EFB007002052F532FC7F582852F83740AF005A7
:103F0B0030E5307002052F532FC7906B7863A201F9
:103F1B00852F8385308263A2017F061231F77406E9
:103F2B002530F530E4352FF52F852D83852E8263D3
:103F3B00A201852F8385308263A2011231DBE4FC61
:103F4B00FDFE907013E0F8A3E0F9A3E0FAA3E02FD5
:103F5B00FFEE3AFEED39FDEC38FCEF2408FFE43EB2
:103F6B00FEE43DFDE43CFC907013122AC0907013EC
:103F7B00E0908040F0907014E0908041F0907015CC
:103F8B00E0908042F0907016E0908043F0908000BB
:033F9B007420F09F
:013F9E002200
:0A3CAC008E2C8F2D8C2E8D2F8B3067
:103CB600908000E030E507906DB27401F0229070BC
:103CC60013E0FCA3E0FDA3E0FEA3E0F5368E358D00
:103CD600348C33E536FFE5355407FEE42FF532EE36
:103CE60034C0F531853282F5837423F00532E5322E
:103CF600700205315331C7F582853183740AF005A8
:103D060032E532700205315331C7906B7863A201F8
:103D160085318385328263A2017F061231F77406EC
:103D26002532F532E43531F531852C83852D8263D4
:103D3600A20185318385328263A2011231DB8F377E
:103D4600EF2532F532E43531F531E5306017852E51
:103D560083852F8263A20185318385328263A20126
:103D6600AF301231F7E53724082530F530FFE4FC93
:103D7600FDFEE5362FF536EE3535F535ED3534F500
:103D860034EC3533F533908040E533F0A3E534F079
:103D9600A3E535F0A3E536F09080007420F0AF3649
:0C3DA600AE35AD34AC33907013122AC05F
:013DB20022EE
:064080008E2D8F2E8D2F06
:10408600908000E030E507906DB27401F0229070E8
:1040960013E0FCA3E0FDA3E0FEA3E0F5358E348D2E
:1040A600338C32E535FFE5345407FEE42FF531EE67
:1040B60034C0F530853182F5837423F00531E5315E
:1040C600700205305330C7F582853083EBF0053139
:1040D600E531700205305330C7906B7863A20185D5
:1040E600308385318263A2017F061231F77406257B
:1040F60031F531E43530F530852D83852E8263A286
:104106000185308385318263A201AF2F1231F774A6
:1041160008252FF52FFFE4FCFDFEE5352FF535EEDE
:104126003534F534ED3533F533EC3532F5329080F0
:1041360040E532F0A3E533F0A3E534F0A3E535F02E
:104146009080007420F0AF35AE34AD33AC32907051
:0441560013122AC056
:01415A002242
:02481C008F40CB
:10481E00908000E030E507906DB27401F022907048
:10482E0013E0FCA3E0FDA3E0FEA3E0F5448E438D70
:10483E00428C41E544FFE5435407FEE42FFFEE347E
:10484E00C0906AEE63A201F5838F8263A201AF402E
:10485E001231F7E4FCFDFEE5442540F544EE354308
:10486E00F543ED3542F542EC3541F541908040E59A
:10487E0041F0A3E542F0A3E543F0A3E544F09080B8
:10488E00007420F0AF44AE43AD42AC4190701312B1
:02489E002AC02E
:0148A00022F5
:063F9F008E2A8F2BAB05FA
:103FA500908000E030E507906DB27401F0229070CA
:103FB50013E0FCA3E0FDA3E0FEA3E0F5318E308D18
:103FC5002F8C2EE531FFE5305407FEE42FF52DEE5D
:103FD50034C0F52C852D82F5837423F0052DE52D50
:103FE5007002052C532CC7F582852C83EBF0052D2B
:103FF500E52D7002052C906B7863A201852C8385D5
:104005002D8263A2017F061231F77406252DF52D49
:10401500E4352CF52C532CC7E52A852D82852C8378
:10402500F0052DE52D7002052C532CC7F582852C46
:1040350083E52BF0052DE52D7002052C532CC7E5E6
:1040450031240AF531E43530F530E4352FF52FE428
:10405500352EF52E908040E52EF0A3E52FF0A3E553
:1040650030F0A3E531F09080007420F0AF31AE3030
:0A407500AD2FAC2E907013122AC07C
:01407F00221E
:104F8600A2AF9220C2AF438E2075D2028F828E834B
:0C4F9600E0FFE4F5D2538EDFA22092AFC2
:014FA20022EC
:104F1A00E5D220E0FBA2AF9220C2AF43D2028F8239
:104F2A008E83EDF075D25063D250A22092AFE5D2B3
:034F3A0020E0FB79
:014F3D002251
:1049A900E4FDED2401FFE433FE124F8674702DF50A
:1049B90082E4346BF583EFF00DBD3FE6E4FDED24B1
:1049C9007FFFE433FE124F8674672DF582E4346964
:1049D900F583EFF074672DF582E43469F583E070AF
:1049E9001B74672DF582E43469F5837420F07468CB
:1049F9002DF582E43469F583E4F080040DBD80BEB1
:104A0900E49069E6F0FDEDFF7E00124F8674E72D14
:0D4A1900F582E43469F583EFF00DBDFEE990
:014A2600226D
:024E36008B2CC3
:104E3800A2AF9220C2AF85A22D53A2FE8E838F828D
:104E480005A28C838D827409123281E52C53A2FE4F
:104E580043A22012328353A2DF852DA2A22092AF53
:014E6800FF4A
:014E69002226
:104FA300A2AF9220C2AF8C838D82EF12328143A2D3
:0C4FB3002012328353A2DFA22092AFFF35
:014FBF0022CF
:024F3E008F27BB
:104F4000A2AF9220C2AFE4F5838D82740612328143
:104F5000E52743A22012328353A2DFA22092AF7F23
:014F6000014F
:014F6100222D
:024F62008F2797
:104F6400A2AF9220C2AFE4F5838D82740A1232811B
:104F7400E52743A22012328353A2DFA22092AF7FFF
:014F8400012B
:014F85002209
:1030AA00A907E7FFA805EF93C3966008403B74FCA5
:1030BA002FFF80F00F08EF93C3966008402B74FB34
:1030CA002FFF80E00F08EF93C3966008401B74FA45
:1030DA002FFF80D00F08EF93D3966008400B74F946
:1030EA002FFF80C01F1F1F1F1FEF54FEF80303F797
:1030FA00E893FC08E893FD08E893FE08E893FF22AA
:10310A0009E993C39D6008402974FB29F980F109F4
:10311A00E993C39E6008401A74FA29F980E209E922
:10312A0093D39F6008400B74F929F980D3191919B0
:10313A001919E9C313C313FF22740093F8ECC39857
:10314A004024701F740193F8EDC3984019701474E9
:0E315A000293F8EEC398400E7009740393F8C8
:10316800EFC39840037F00227F0122EDF8E6F008C4
:10317800A3DFFA22EDF8E0F608A3DFFA22E0A36362
:10318800A201F0A363A201DFF475A2002263A201E9
:10319800F0A363A20122E0A363A201F0A363A2014A
:1031A800E0A363A201F0A363A201E463A201F0A378
:1031B80063A201DFE175A20022E0A363A2016DFE14
:1031C800936CFDEE058393FC158363A201DFEA751A
:1031D800A200227F00E493A363A201F00F600CA376
:1031E800E583C2E3F58363A20180EA75A20022E0C9
:1031F800A363A201F0A3E583C2E3F58363A201DF21
:10320800EE75A20022E0A363A201F0A3E583C2E465
:10321800D2E3F58363A201DFEC75A20022E0A36389
:10322800A201F0A3E58344F8C2E5F58363A201DFB8
:10323800EC75A20022E583C2E3F583E0A363A20153
:10324800F0A363A201DFEE75A20022E583C2E4D2F7
:0A325800E3F583E0A363A201F0A3F5
:1032620063A201DFEC75A20022E58344F8F583E056
:10327200A363A201F0A363A201DFEE75A20022F90B
:1032820022C002C004C00612FFF0D006D004D00251
:013292002219
:1045FD004572724C656E210A000A496E49503A00A7
:10460D00205544502054696D654750530A00200AC7
:10461D00444154414752414D3A20002043414E20E0
:10462D0054696D654750530A00205472617373537A
:10463D00656E644552520A000ACEF8C4EBE8EDFBF4
:10464D0043414E210A000A45727241647243414E44
:10465D003A00205265496E69742043414E0A00208C
:10466D0043414E283029203E20544F210A0020542A
:0C467D005520300A0020545520310A005E
:03001E00E4FF22DA
:104ECB00C2A9438902758C48758A4875D90475DB6C
:104EDB004875DC4875DD4875DE48E4F5E9F5F9D22F
:084EEB00D9C2DAD28CD2DE221A
:104E9D00C2D9906EDBE07013E5E92419F5EB30D73C
:104EAD0006E5F904F5FB2285F9FB22E5E924C8F5B1
:0E4EBD00EB30D706E5F904F5FB2285F9FB2260
:104D3E00C2D9906EDBE0702C302D16E5E92432F5E9
:104D4E00EB30D707E5F904F5FB800385F9FBC22D9F
:104D5E0022E5E92405F5EB30D706E5F904F5FB224B
:104D6E0085F9FB22E5E92432F5EB30D706E5F904A7
:074D7E00F5FB2285F9FB2281
:104EF300124ECB906EDBE0C3946450061249251228
:104F03004E9D12504CD22CE4F556906FF3F0F545BC
:074F1300F55AC22DF55822EA
:104D8500EF24FCF545D3940D4010200B077E457F9D
:104D9500FD123EB7E4F545D22A22906BB363A2011A
:104DA500906FE363A201AF45123185C22A200B0D36
:0E4DB5007E467F067C6B7DB3AB45123CAC2284
:0F501200D3EF6480948D5006E55A70028F5A22B6
:10262E0020D903022703202C03022703E55A604A10
:10263E0090683E540FFF7D4712317CE54764017070
:10264E001E906846E0B4FF0ED22E200B127E467FFF
:10265E000D123EB78009302E06E4F55A02270312FA
:10266E004E9D124B7E200B0D7E467F1B7C687D3E61
:10267E00AB5A123CACE4F55A807BE5456043906F53
:10268E00E7E02405F527D3940D4007E4F545D22A5B
:10269E008063906FE3E527540FFF7D4712317CE591
:1026AE004730E702D22DE547B40109302E06E54A40
:1026BE0064016003124B7E124E9DE4F545D22A80D2
:1026CE0034E557601E906EC7540FFF7D4712317C64
:1026DE00E547B40103202E03124B7E124E9DE4F506
:1026EE0057801220110C906EDBE0C39464500312DD
:1026FE004225124E9D123A3B8F27EF700302281D82
:10270E00124D3EE4F558E547B4010CD22E200B07CE
:10271E007E467F28123EB7E559C394C8501B30033E
:10272E001874DC2559F582E4346EF583E5272559B6
:10273E00F5597D47AF27123173300121E54720E768
:10274E001C906DB37D47AF27123173AF2712439A9A
:10275E00EF700A200B077E467F36123EB7E54754D0
:10276E0081600302281DE527D3940D4010300B0322
:10277E0002281D7E467F45123EB702281DE549D32D
:10278E009407401F300B0302281D90693F7D47AF11
:10279E00271231737E467F537C697D3FAB27123CF7
:1027AE00AC806CE51330E66290700EE0FF904C0F3B
:1027BE0093FE547F65477052EFA3936549704B901B
:1027CE00700EE0C313FF24F5F582E4346FF583E059
:1027DE00703853133F90700EE0FD74872513F58209
:1027EE00E43461F583EEF0ED904C1093FE74882581
:1027FE0013F582E43461F583EEF074F52FF582E47F
:10280E00346FF5837401F0431340AF27122BFE3063
:10281E000E1A300015906EDBE0C39464500C055810
:10282E00E55894F04004C2AF80FEC20E20020302AF
:10283E002932E5566031D394014004155680289014
:10284E006FF3E004F0E0D39403400D200B077E46B7
:10285E007F5F123EB7124EF3200B077E467F6C123F
:10286E003EB7E4F556D22C302B43E557703F906EB1
:10287E00C704F0A37408F0A37480F0A37401F0A34E
:10288E007406F0906FDEE0906ECCF0906FDFE0900B
:10289E006ECDF0906FE0E0906ECEF0906FE1E09034
:1028AE006ECFF0E4A3F0A3F075570BC22B30297254
:1028BE00906FDCE07035E5577031906EC77442F062
:1028CE00A37408F0906FDDE0906EC9F0906FE2E0B7
:1028DE00906ECAF0A37401F0755706200B077E4662
:1028EE007F7B123EB7906FDCE004F0906FDCE0640B
:1028FE0002702FE557702B906EC77402F0A3740808
:10290E00F0906FDDE0906EC9F0A3F0A37401F07546
:10291E005706200B077E467F82123EB7906FDCE093
:09292E0004F0C202120026C200EE
:01293700227D
:104E6A00E559602CE4906CAFF0A3E559F0906EB46C
:104E7A00E0906CB1F0A37419F0906EDC63A201901B
:104E8A006CB363A201AF59123185E4F5597F01224F
:034E9A007F002274
:0B502100302A05C22A7F01227F0022F6
:0100210022BC
:06504600E4F559F54522D6
:0A502C00E490693FF0A3F0A3F02226
:104BE0002043616E457247495400200A00457272A5
:104BF0004C656E43616E21000A002043616E457270
:104C000072434821000A205265714572722100C426
:104C100000C401C402C403C404C405C406C407C854
:104C200000C801C802C803C804C805C806C807C22E
:104C300000C201C202C203C204C205C206C207000A
:014C40000073
:103A3B00E59B541F6020200B1A7E4B7FE0123EB794
:103A4B00E59B541FFF7E007D03123F9F7E4B7FEA59
:103A5B00123EB7E4F59BE5BA30E010E4F5B375B16F
:103A6B0080F5B2D22CF556906FF3F0E5CFF47003DE
:103A7B00023B90752901E4F528E5CFF45529700335
:103A8B00023B7EE528C454F0F5B1E5B2547F6420C7
:103A9B006003023B4FE5B3540FF54B85BC47E5BDC7
:103AAB00541FFF131313541FFFE5BD54E044184F6D
:103ABB00F548E5BDC43354E0FFE5BE131313541FA3
:103ACB004FF549E5BEC43354E0FFE5BF1313135460
:103ADB001F4FF54A85A34C85A34D85A34E85A34F58
:103AEB0085A35085A35185A35285A353E4F5B2203A
:103AFB00110CE547547EB5470575B350800375B37C
:103B0B00D0E54B700AE547547EB547037F00223062
:103B1B001108E54730E7037F0022E54BD3940840BB
:103B2B001D200B177E4B7FED123EB7AF4B7E007DFA
:103B3B0003123F9F7E4B7FF8123EB77F0022E54B6F
:103B4B002405FF22E5B2549F6023200B207E4B7F80
:103B5B00FA123EB7AFB27E007D03123F9FAFB37E2A
:103B6B00007D03123F9F7E4B7FF8123EB7E4F5B208
:103B7B0075B3D0E52925E0F5290528E528C3940878
:073B8B005003023A847F00A1
:013B92002210
:104B7E00906EDBE0C39464505675B180E4F5B3F5E6
:104B8E00B28547BCE549C4135407FFE54854E04FCE
:104B9E00F5BDE54933333354F8FFE54AC4135407E2
:104BAE004FF5BEE54A33333354F8F5BF854CA38534
:104BBE004DA3854EA3854FA38550A38551A3855242
:104BCE00A38553A3E54B540F2450F5B375560AC273
:024BDE002C2287
:1042250075B190E5B220E613200B107E4C7F051288
:104235003EB7AFB27E007D03123F9FE4F5B3F5B202
:1042450074872513F582E43461F583E0701B907063
:104255000EE0FFC31324F5F582E4346FF583E070B7
:10426500054313808003431340E51330E615E4F559
:104275001390700EE02402F0E0904C0F93700490C0
:10428500700EF0E51330E72190700EE0FF904C0FB3
:1042950093F5BCE4F5BDEFA393FF33333354F8F541
:1042A500BE75BF78431340803674872513F582E4C5
:1042B5003461F583E0F5BCE4F5BD74882513F5821A
:1042C500E43461F583E0FF33333354F8F5BE75BF4D
:1042D5007805130513E513C394324003E4F513750C
:0342E500B35022B1
:09503600EF6003C29622D296221B
:1049250043AB01C2E8C2EAE4FFEFC454F0F5B1C3FA
:10493500EF64809488500575B3D08003E4F5B3E443
:10494500F5B2F5BCF5BDF5BEF5BFF5C4F5C5F5C6C3
:10495500F5C7F5A3F5A3F5A3F5A3F5A3F5A3F5A36E
:10496500F5A30FBF0EC3906EDBE0FE25E0F5B47531
:10497500B50C75B66C75A11275AB0275C13E75C3E4
:10498500FF75C203E490700EF0751380FF7F1990D8
:104995006FF5E4F0A3DFFCE4FF7F32906187E4F07C
:0349A500A3DFFC91
:0149A80022EC
:101141005452414E5A004D415842005254530044AA
:10115100454C4159004D4F4445004B5000545500FA
:1011610043414E004B565400415400444952004300
:10117100414E4D4F4E00475254494D45005449543C
:1011810053005453494E5600003E2A2C312CCFE0D7
:10119100F0E0ECE5F2F0FB20F3EFF0E0E2EBFFFE34
:1011A100F9E5E3EE20EAEEEDF2F0EEEBEBE5F0E04F
:1011B10020CACF20C8F1E5F2FC0A003E4C2C6B306E
:1011C100312C25732C43EAEEF0EEF1F2FC20EDE038
:1011D10020F8E8EDE52043414E2C30202D2035301C
:1011E10030EAE1283530EC292C31202D203530EA48
:1011F100E128353030EC290A0030202D20353030FF
:10120100EAE1283530EC290031202D203530EAE1A2
:1012110028353030EC29003E532C6B30322C2562BE
:10122100752CCCE0EAF12E20E0E4F0E5F120E1EBD1
:10123100EEEAE020D2D128302D38290A003E532C85
:101241006B30332C2562752CCCE0EAF12E20E0E4E2
:10125100F0E5F120E1EBEEEAE020D2C8D228302D12
:1012610038290A003E532C6B30342C2562752CCC66
:10127100E0EAF12E20E0E4F0E5F120E1EBEEEAE036
:1012810020D2D328302D38290A003E422C63303138
:101291002C2562752CC2F2EEF0E8F7EDFBE920EAAD
:1012A100EEEDF2F0EEEBEBE5F020EDE020F8E8ED0D
:1012B100E50A003E2A2C312CCFE0F0E0ECE5F2F01B
:1012C100FB20EFF0EEF2EEEAEEEBE020C3F0E0ED12
:1012D100E8F220EFEE20EFEEF0F2F320525332333A
:1012E100320A003E432C61636B2C25732CCFEEF048
:1012F100FFE4EEEA20C0D4C10A00312DD2D128305A
:101301002B312920322DD2C8D228302920332DD299
:10131100D320342DD2C8D228312920352DD2D1283D
:10132100322B332920382DD2C8C8003E4C2C6B30CB
:10133100352C256C752CD1EAEEF0EEF1F2FC20EEA5
:10134100E1ECE5EDE020EDE020EFEEF0F2F32C3101
:1013510030302C3230302C3330302C3630302C3190
:101361003230302C323430302C343830302C393665
:1013710030302C31393230302C33383430302C3558
:10138100373630302C3131353230300A003E532C73
:101391006B30362C2562752CCDEEECE5F020CACFF2
:1013A100200A003E422C6730312C2562752CCCE09E
:1013B100E3E8F1F2F0E0EBFC0A003E422C67303248
:1013C1002C2562752CC8EDE2E5F0F2E8F0EEE2E0E2
:1013D100F2FC20E7EDE0F7E5EDE8FF20D2D10A00CD
:1013E1003E422C6730332C2562752CC7E0EFF0E0CC
:1013F100F8E8E2E0F2FC20E2F0E5ECFF20F1E5F0B4
:10140100E2E5F0E00A003E422C6730342C2562759B
:101411002CC2FBF1F2E0E2EBFFF2FC20525453202C
:10142100EFF0E820EFE5F0E5E4E0F7E50A003E53F0
:101431002C6730352C2562752CC7E0E4E5F0E6EA2F
:10144100E020EFE5F0E5E4E0F7E820EFEEF1EBE591
:101451002052545320282A3130ECF1290A003C2132
:10146100003C6B30313D003C6B30323D003C6B3019
:10147100333D003C6B30343D003C6330313D003C3A
:101481006B30353D003C6B30363D003C6730313DC3
:10149100003C6730323D003C6730333D003C6730F3
:1014A100343D003C6730353D000ACFE5F0E5E4E02E
:1014B100F7E03A2000544949204379636C650A00FA
:1014C1005453204379636C650A0054530A0054490C
:1014D100540A005455204F4B0A0054552044696169
:1014E100670A005455205265710A00205455205452
:1014F100696D654F5554210A000ACFF0E8E5EC3AD1
:1015010020000A4352432045525221000AD7F3E6F4
:10151100EEE920EDEEECE5F020CACF21000A52659C
:101521007154533120000A52657154533520000A19
:1015310052657154495420000ACFF0E8EDFFF2E002
:1015410020EAEEECE0EDE4E020D2D320002020D22E
:10155100D320E7E0EDFFF2EE210A000ACDE520EF0E
:10156100EEEDFFEB20F2E8EF20EFE0EAE5F2E0211B
:101571000A0000112332465765748C9DAFBECADB49
:10158100E9F810013322564775649C8DBFAEDACB62
:10159100F9E82130021367764455ADBC8E9FEBFA12
:1015A100C8D93120120377665445BDAC9E8FFBEA42
:1015B100D8C94253617004152736CEDFEDFC8899F6
:1015C100ABBA5243716014053726DECFFDEC988922
:1015D100BBAA6372405125340617EFFECCDDA9B8D2
:1015E1008A9B7362504135241607FFEEDCCDB9A802
:1015F1009A8B8495A7B6C2D3E1F008192B3A4E5FB6
:101601006D7C9485B7A6D2C3F1E018093B2A5E4FE1
:101611007D6CA5B48697E3F2C0D129380A1B6F7E91
:101621004C5DB5A49687F3E2D0C139281A0B7F6EC1
:101631005C4DC6D7E5F48091A3B24A5B69780C1D75
:101641002F3ED6C7F5E49081B3A25A4B79681C0DA1
:101651003F2EE7F6C4D5A1B082936B7A48592D3C51
:101661000E1FF7E6D4C5B1A092837B6A58493D2C81
:101671001E0F0089129B24AD36BF48C15AD36CE5B9
:101681007EF78108931AA52CB73EC940DB52ED6461
:10169100FF76028B109926AF34BD4AC358D16EE74D
:1016A1007CF5830A9118A72EB53CCB42D950EF6641
:1016B100FD74048D169F20A932BB4CC55ED768E12D
:1016C1007AF3850C971EA128B33ACD44DF56E96021
:1016D100FB72068F149D22AB30B94EC75CD56AE30D
:1016E10078F1870E951CA32AB138CF46DD54EB6201
:1016F100F97008811A932CA53EB740C952DB64EDFD
:1017010076FF89009B12AD24BF36C148D35AE56CE0
:10171100F77E0A8318912EA73CB542CB50D966EFCC
:1017210074FD8B029910AF26BD34C34AD158E76EC0
:10173100F57C0C851E9728A13AB344CD56DF60E9AC
:1017410072FB8D049F16A920BB32C54CD75EE168A0
:10175100F37A0E871C952AA338B146CF54DD62EB8C
:1017610070F98F069D14AB22B930C74ED55CE36A80
:10177100F1780008040C020A060E0109050D030B9D
:10178100070FFF1141FF1147FF114CFF1150FF11CE
:1017910056FF115BFF115EFF1161FF1165FF1169BA
:1017A100FF116CFF1170FF1177FF117EFF1183FF95
:0217B10011899C
:104FDA00EF540F90177393FEC454F0FEEFC4540FAE
:044FEA00932EFF22E1
:0300230002444A4A
:0B444A00C0E0C083C082C0D075D01855
:10445500309852C298755E01AF9920164820120B0C
:10446500EF64027040D212D291803A301A04C21A17
:104475008024BF0904D21A802CBF0205530B80800B
:1044850024BF0312906614E50BF0630B80530B8079
:10449500C212C291800F7437250BF582E43466F59C
:1044A50083EFF0050B30992B301326906185E0FFE3
:1044B500E50CC39F4008C213D21DC2908013D29051
:1044C500AF0C050C74372FF582E43467F583E0F5FE
:0344D50099C299F0
:0944D800D0D0D082D083D0E032B4
:103B93007BFF7A11798A122334906EDBE0701475FF
:103BA3002FFF7530117531FA7BFF7A1179BC12231F
:103BB300348012752FFF7530127531097BFF7A112E
:103BC30079BC1223347BFF7A127918906186E0F571
:103BD3002F1223347BFF7A12793E906101E0F52F97
:103BE3001223347BFF7A127965906100E0F52F127E
:103BF30023347BFF7A12798BA211E433F52F12233E
:103C0300347BFF7A1279B4122334752FFF75301287
:103C13007531FB7BFF7A1279E4122334906838E024
:103C2300FEA3E0FFC3E49FFFE49EFEAB07FA3395D8
:103C3300E0F9F87F007E8C7D0A7C00122A0F8F3218
:103C43008E318D308C2F7BFF7A13792C1223347BAA
:103C5300FF7A13798E906403E0F52F1223347BFFF0
:103C63007A1379A4A21EE4336401F52F1223347B63
:103C7300FF7A1379BBA219E433F52F1223347BFFA8
:103C83007A1379E1A214E433F52F1223347BFF7AFC
:103C9300147907A21BE433F52F1223347BFF7A1424
:093CA300792F85092F1223342228
:103766007E147F5F124797EF4E70037F0122E4902D
:103776006EDBF07E147F62124797EF4E6015124F94
:10378600C0BF3106906EDB740AF0BF3206906EDB66
:103796007464F07E147F68124797EF4E600A124CED
:1037A60041906186EFF080069061867402F07E1487
:1037B6007F6E124797EF4E600A124C41906101EFFF
:1037C600F080069061017402F07E147F74124797B0
:1037D600EF4E600A124C41906100EFF08006906156
:1037E600007402F07E147F7A124797EF4E600D1236
:1037F6004C41EC4D4E4F24FF92118002C2117E14B3
:103806007F80124797EF4E6023124C41A804A9050A
:10381600AA06AB077F007E8C7D0A7C00122A0F1257
:103826002AA1906838EEF0A3EFF0800A9068387409
:10383600FFF0A374DCF07E147F86124797EF4E608C
:103846000A124C41906403EFF08006906403740101
:10385600F07E147F8C124797EF4E600E124FC0EF2A
:1038660024D0640124FF921E8002C21E7E147F9221
:10387600124797EF4E600C124FC0EF24D024FF92F0
:10388600198002C2197E147F98124797EF4E600C7A
:10389600124FC0EF24D024FF92148002C2147E146B
:1038A6007F9E124797EF4E600C124FC0EF24D02434
:1038B600FF921B8002C21B7E147FA4124797EF4E15
:0E38C6006007124C418F098003E4F5097F0072
:0138D40022D1
:102EA100E4F527E52775F003A42483F582E43417BC
:102EB100F583E493FB740193FA740293F9122938B0
:102EC10070030230A9E4F529F52AF528746725284D
:102ED100F582E43469F583E0FF70030230A4E5274D
:102EE10075F003A42483F582E43417F583E493FB9E
:102EF100740193FA740293F985298275830012296A
:102F010051FEEFB50608752A01052902309FE52A11
:102F1100700302309FEE600302309AE527B40F0080
:102F210040030230A4902F2DF8282873022F5A0253
:102F31002FA1022FDA022FDF0230A4023037023034
:102F4100A402300A0230A40230A402306402308E9E
:102F51000230920230A402309674672528F9E434D5
:102F610069FA7B01C0031B8B32753300753400E4B1
:102F7100F535D00312343B8F2E8E2D8D2C8C2BAB3F
:102F81002EAA2DA92CA82B7F007E8C7D0A7C0012F5
:102F91002A0F122AA1906838EEF0A3EFF00230A4B4
:102FA10074672528F582E43469F583E024D09061C3
:102FB10086F074682528F582E43469F583E024D02D
:102FC100906101F074692528F582E43469F583E0A4
:102FD10024D0906100F00230A4D21B0230A47467A7
:102FE1002528F9E43469FA7B01C0031B8B32753360
:102FF10000753400E4F535D00312343B8F2E8E2D4D
:103001008D2C8C2B8F090230A474672528F9E434A8
:1030110069FA7B01C0031B8B32753300753400E400
:10302100F535D00312343B8F2E8E2D8D2C8C2B90A9
:103031006EDBEFF0806D74672528F9E43469FA7B63
:1030410001C0031B8B32753300753400E4F535D0B4
:103051000312343B8F2E8E2D8D2C8C2B906403EF1D
:10306100F0804074672528F9E43469FA7B01C003D4
:103071001B8B32753300753400E4F535D0031234FF
:103081003B8F2E8E2D8D2C8C2BD21E8016D2118033
:1030910012D214800EC219800AE4F52AF5290528F6
:0830A100022ECD0527022EA42A
:0130A9002204
:10329300C229C21CC218C217C215E4906837F0C213
:1032A3001F9066167405F0C22BE4F508FF7F40906B
:1032B30061B9E4F0A3DFFCE4FF7F20906617E4F03C
:1032C300A3DFFCE4FF74042FF582E43466F583E4A2
:1032D300F0740C2FF582E43466F583E4F00FBF0835
:1032E300E4E4F50DF50EF512F511906302F0906329
:1032F30001F0C213C21DC216C212C21AF50C9061AC
:1033030085F0F509F50BF55EC210C21B90683874A1
:10331300FFF0A374F4F0E4906403F0C21EC211C280
:1033230014D219906EDBF0123766EF6003122EA1F0
:10333300E4F5137E617F87906186E0F513E513C39F
:1033430094014007E513D394084003E4F513E51310
:1033530060220FEFAC0670010E14F5828C8374C4E7
:10336300F015130FEFAC0670010E14F5828C83E594
:1033730013F080DA906101E0F513E513C394014083
:1033830007E513D394084003E4F513E51360220F14
:10339300EFAC0670010E14F5828C8374C8F015131C
:1033A3000FEFAC0670010E14F5828C83E513F080E9
:1033B300DA906100E0F513E513C394014007E513C8
:1033C300D394084003E4F513E51360220FEFAC0632
:1033D30070010E14F5828C8374C2F015130FEFACD9
:1033E3000670010E14F5828C83E513F080DA0FEF7B
:1033F300AC0670010E14F5828C83E4F08F828E8309
:10340300F0F513C2ADF5C9D2CDD2CCC2C9C2CAF54B
:10341300CDF5CC906838E0F5CBA3E0F5CA85CBCDEC
:1034230085CACCD29ED29CD2CAC2ACC298C299756C
:07343300B81075B710D2AC10
:01343A00226F
:104FEE00E5106FFF90167393650FF510EF90157324
:034FFE0093F50F19
:01500100228C
:0242E8008F2D18
:1042EA00E4FC752E61752F02F510F50FFDEDC395EF
:1042FA002D5017052FE52FAE2E7002052E14F582CC
:10430A008E83E0FF124FEE0D80E3052FE52FAE2ED0
:10431A007002052E14F5828E83E510F0852F8285B2
:10432A002E83E50FF0052D052D7E677F37752E61EB
:10433A00752F028F828E837402F00FBF00010E0C5C
:10434A00E4FDEDC3952D5038852F82852E83E0F943
:10435A0064026008E964036003B9090D8F828E83E1
:10436A007409F00FBF00010E0C8F828E83E9F00FE3
:10437A00BF00010E0C052FE52F7002052E0D80C21D
:0F438A008F828E837403F00FBF00010E0CAF04FF
:014399002201
:03504C00C2162267
:104DC3008F2C201335AF2C1242E8906185EFF02031
:104DD3000B127E147FAA123EB77E617F02E4FBAD05
:104DE3002C124080301B057F01125036E509600309
:0B4DF300F55B22E4F50CD213D29922EC
:022BFE008F281E
:102C0000E54724BE7003022E4924FA7003022DC149
:102C100024046003022EA0E54830E703022CC530EF
:102C20000C077E147FB6123EB7E54A6068E549C3DB
:102C300094024003022EA0E5497007E54A14F529E5
:102C40008006E54A241FF529E52975F004A424032C
:102C5000F582746335F0F5837D4C7F04123173E5A2
:102C60002975F004A42401F582746235F0F5837DA2
:102C7000507F0412317374F92549F582E43461F50B
:102C8000837481F074B92529F582E43461F5837485
:102C900001F0D21722300C077E147FC1123EB774A8
:102CA000042549F582E43466F5837401F0E549753D
:102CB000F004A42417F582746635F0F5837D4C7F0B
:102CC0000412317322E54B64086003022EA0E5492B
:102CD000C394044003022EA0300C077E147FCB1255
:102CE0003EB7752801E54A5407FFE528A807088084
:102CF00002C333D8FCF5287408250EF50EB50D0671
:102D00007408250DF50DE54A547FFFE549C4335499
:102D1000E02FFE7400250EF582E43460F583EEF0BA
:102D2000E54AC394805022EF131313541FFFE54963
:102D300025E025E02F2417F582E43466F583E0FFD3
:102D4000E528F4FEEF5EF0802EE54A547FFF131372
:102D500013541FFFE54925E025E02F2417F582E4F1
:102D60003466F583E04528F07400250EF582E434DE
:102D700060F583E04480F07401250EF582E4346050
:102D8000F5837D4C7F04123173E551FEE550FF7CE5
:102D9000007D0A12297EEF7405250EF582E4346069
:102DA000F583EFF07406250EF582E43460F583E5D3
:102DB00052F07407250EF582E43460F583E553F094
:102DC00022300C077E147FCF123EB7E54A54E064F0
:102DD000407003022EA0E54A547FF529E549701D95
:102DE000E5291313543FFF7401A807088002C33379
:102DF000D8FC4211906301E04511F08024E549645C
:102E0000016003022EA0E5291313543FFF7401A8AB
:102E100007088002C333D8FC4212906302E04512D7
:102E2000F0E54975F020A47C002529FFEC35F0FE83
:102E3000EF25E0FFEE33FE74042FF58274643EF557
:102E4000837D4CAF4B12317322E54AB40113300C31
:102E5000077E147FD4123EB7E54D04906FF4F0C2A4
:102E600029E54AB40216240CF582E43466F583E5BC
:102E70004DF0300C077E147FDB123EB7E54AB403F9
:102E80001F240CF582E43466F583E54DF0300C0721
:102E90007E147FE4123EB7302906906FDC7402F096
:012EA000220F
:10002600906403E070030208E130002F050A906631
:1000360016E0600214F0906837E0600214F0C20027
:10004600302918906184E004F0E0D3940A400C3023
:100056000C077E147FEC123EB7C229E55BB401099A
:10006600E4F55BF50CD213D29930130DE50AD3945F
:10007600064009C213D21D8003E4F50A301D0AC2E8
:100086001D301B05E4FF12503630130302053DE513
:100096005B600302053D201E0620150302053DC2D6
:1000A60015301F29C21FE4906102F0A37408F09076
:1000B6006403E0906104F0906615E0906105F0A39A
:1000C60074FEF0A3748FF07F06124DC322906FF476
:1000D600E0FF6025E4906102F0A37408F0906403E9
:1000E600E0906104F0A37483F0A3EFF0E4A3F09032
:1000F6006FF4F07F06124DC322E50E650D70030204
:100106000200906837E060030202DAE50D2408F584
:1001160028E4906102F0A37408F0906403E0906113
:1001260004F0A374F0F0A37406F0A37491F07406BF
:100136002528F582E43460F583E0906108F07407C1
:100146002528F582E43460F583E0906109F07401B6
:100156002528F582E43460F583E090610AF07402A4
:100166002528F582E43460F583E090610BF0740392
:100176002528F582E43460F583E090610CF0740480
:100186002528F582E43460F583E090610DF0740073
:100196002528F582E43460F583E0FF547FFEC3949E
:1001A60040500BEFC454F00490610EF080167400BA
:1001B6002528F582E43460F583E0FFC454F0240575
:1001C60090610EF074002528F582E43460F583E032
:1001D600FFEEC4540F90610FF0EF5480FF740525B5
:1001E60028F582E43460F583E02F906110F0906882
:1001F600377414F07F0F124DC32230186AE49061F1
:1002060002F0A37408F0906403E0906104F0A37414
:1002160041F0A37420F0752A61752B07E4F5287464
:10022600172528F582E43466F583E0F529301906AA
:10023600FF124FDA8F29852B82852A83E529F0F470
:10024600FFE5822408F582E43583F583EFF0052B7C
:10025600E52B7002052A0528E528C3940840C07FCF
:1002660015124DC3C21822301C6AE4906102F0A335
:100276007408F0906403E0906104F0A37445F0A361
:100286007420F0752A61752B0775280874172528C0
:10029600F582E43466F583E0F529301906FF124F3E
:1002A600DA8F29852B82852A83E529F0F4FFE582FA
:1002B6002408F582E43583F583EFF0052BE52B70F2
:1002C60002052A0528E528C3941040C07F15124D63
:1002D600C3C21C222017030203DD9061FAE0FF90DF
:1002E60061F9E04F5401D3940050030203DDE4F5B5
:1002F6002874B92528F582E43461F583E070030299
:1003060003CF74B92528F582E43461F583E4F090CF
:100316006102F0A37408F0906403E0906104F0A316
:1003260074F0F0A37403F0A37491F0E528C4540F9D
:100336002408A3F0E528540FA3F0E52825E025E0DE
:10034600F5282401F582E43462F583E090610AF031
:1003560074022528F582E43462F583E090610BF09F
:1003660074032528F582E43462F583E090610CF08D
:1003760074042528F582E43462F583E090610DF07B
:10038600E4A3F074032528F582E43463F583E09052
:10039600610FF074042528F582E43463F583E09058
:1003A6006110F074052528F582E43463F583E09046
:1003B6006111F074062528F582E43463F583E09034
:1003C6006112F07F11124DC3220528E528C394401F
:1003D60050030202F7C217906616E0704130143ED1
:1003E6007478F0E4906102F0A37408F0906403E07E
:1003F600906104F0A374F0F0E4A3F0A37490F0A36A
:100406007408F0E4A3F0A3F0A3F0A3F0A3F0A3F024
:10041600A3F0A3F0A3F0A3F07F11124DC322E508C9
:10042600C39404506FE50825E0FF7403A80708800D
:1004360002C333D8FCF528551165287053E528F416
:100446005211E4906102F0A37408F0906403E09006
:100456006104F0A374F0F0A37402F0A37491F0E5C4
:10046600082420A3F0E50833333354F875F002A4CA
:100476002404F582E5F03464F58363A201906109F2
:1004860063A2017F101231857F17124DC305082222
:100496000508808AE508C394085076E50824FC25FB
:1004A600E0FF7403A807088002C333D8FCF528557B
:1004B6001265287058E528F45212E4906102F0A300
:1004C6007408F0906403E0906104F0A374F0F0A364
:1004D6007402F0A37491F0E50854032440A3F0E5F8
:1004E6000833333354F875F002A42404F582E5F09A
:1004F6003464F58363A20190610963A2017F10123F
:1005060031857F17124DC305085308072205088059
:1005160083E4F508201E20E4906102F0A37408F03D
:10052600906403E0906104F0A37490F0E4A3F0A358
:10053600F07F06124DC322906614E0FF7003020896
:10054600E1F529E4F0200B1F7E147FFA123EB7E591
:100556002954802437F582E43466AF82FEE52954B7
:100566007FFDE4FB124080E52970030208E1E529DE
:100576005480FF2437F582E43466AD82F52A8D2B4C
:10058600E4F510F50F8F28E528C395295018052B9B
:10059600E52BAE2A7002052A14F5828E83E0FF123F
:1005A6004FEE052880E1E50F4510600E300B030283
:1005B60008E17E157F03123EB722E52954802437D1
:1005C600F582E43466AF82F52A8F2B7402252BF56B
:1005D6002BE4352AF52A852B82F583E0FF90640308
:1005E600E0FEEF6E600E300B030208E17E157F0D14
:1005F600123EB722052BE52B7002052AF582852AC5
:1006060083E0FFB43003D21522EF640170030208C1
:10061600E1EF64187037906605E0FF906604E04FDE
:10062600600CD218200B077E157F1E123EB790660F
:1006360007E0FF906606E04F70030208E1D21C3027
:100646000B030208E17E157F27123EB722852B8217
:10065600852A83E0B41915200B077E157F30123EDC
:10066600B7906301E0F511A3E0F51222852B828590
:100676002A83E0FF54F064F0600302076990661570
:10068600EFF0052BE52B7002052AF582852A83E01B
:10069600FF64807033052BE52B7002052AF58285F1
:1006A6002A83E0644060030208E1D21F052BE52B94
:1006B6007002052AF582852A83E064086003020831
:1006C600E1D214906616F022EFB40127052BE52B34
:1006D6007002052AF582852A83E0644F60030208CA
:1006E600E1906837E070030208E17408250DF50D06
:1006F600E4F022852B82852A83E060030208E10567
:100706002BE52B7002052AF582852A83E064426078
:10071600030208E1052BE52B7002052AF582852ADE
:1007260083E0906FDEF0052BE52B7002052AF5823B
:10073600852A83E0906FDFF0052BE52B7002052AF2
:10074600F582852A83E0906FE0F0052BE52B700299
:10075600052AF582852A83E0906FE1F0D22BC21438
:10076600D21F22852B82852A83E0FF64116008EF61
:10077600641260030208BFE529547F640E60030219
:1007860008BF200B077E157F39123EB730290E3081
:100796000B030208E17E157F4E123EB722852B829F
:1007A600852A83E0540314F529052BE52B700205F1
:1007B6002AF582852A83E0F52830E709E4906FDD83
:1007C600F0906FE2F0E52830E60BE4906FDDF090F4
:1007D6006FE27410F0E52830E50B906FDD7401F0E0
:1007E600E4906FE2F0E52830E40C906FDD7401F0E0
:1007F600906FE27410F0E52830E30B906FDD740221
:10080600F0E4906FE2F0E52830E20C906FDD7402C0
:10081600F0906FE27410F0E52830E10B906FDD7414
:1008260003F0E4906FE2F0E52830E00C906FDD74A1
:1008360003F0906FE27410F07402252BF52BE4356B
:100846002AF52A852B82F583E0F52830E700E5288E
:1008560030E607906FE2E02402F0E52830E50790E5
:100866006FE2E02404F0E52830E407906FE2E0242C
:1008760006F0E52830E307906FE2E02408F0E5286B
:1008860030E207906FE2E0240AF0E52830E10790B5
:100896006FE2E0240CF0E52830E007906FE2E024F8
:1008A6000EF0906FE2E02529F0D229E4906184F001
:1008B600906FDCF0906FF4F022200B1F7E157F5CAA
:1008C600123EB7E52954802437F582E43466AF82B8
:0B08D600FEE529547FFDE4FB1240808A
:0108E10022F4
:10457D000217B3E493A3F8E493A34003F68001F28A
:10458D0008DFF48029E493A3F85407240CC8C3333F
:10459D00C4540F4420C8834004F456800146F6DF0E
:1045AD00E4800B010204081020408090503FE47E0F
:1045BD00019360BCA3FF543F30E509541FFEE49303
:1045CD00A360010ECF54C025E060A840B8E493A3CA
:1045DD00FAE493A3F8E493A3C8C582C8CAC583CAF5
:1045ED00F0A3C8C582C8CAC583CADFE9DEE780BEAD
:01504500006A
:10293800BB010689828A83E0225002E722BBFE029D
:09294800E32289828A83E49322D0
:10295100BB010CE58229F582E5833AF583E022503B
:1029610006E92582F8E622BBFE06E92582F8E22285
:0D297100E58229F582E5833AF583E493229F
:10297E00BC000BBE0029EF8DF084FFADF022E4CC3D
:10298E00F875F008EF2FFFEE33FEEC33FCEE9DEC06
:10299E00984005FCEE9DFE0FD5F0E9E4CEFD22ED4C
:1029AE00F8F5F0EE8420D21CFEADF075F008EF2F96
:1029BE00FFED33FD4007985006D5F0F222C398FD87
:0529CE000FD5F0EA2224
:1029D30075F008758200EF2FFFEE33FECD33CDCCBB
:1029E30033CCC58233C5829BED9AEC99E58298403E
:1029F3000CF582EE9BFEED9AFDEC99FC0FD5F0D61B
:102A0300E4CEFBE4CDFAE4CCF9A88222B800C1B944
:102A13000059BA002DEC8BF084CFCECDFCE5F0CB82
:102A2300F97818EF2FFFEE33FEED33FDEC33FCEBBB
:102A330033FB10D703994004EB99FB0FD8E5E4F976
:102A4300FA227818EF2FFFEE33FEED33FDEC33FC63
:102A5300C933C910D7059BE99A4007EC9BFCE99A57
:102A6300F90FD8E0E4C9FAE4CCFB2275F010EF2F9C
:102A7300FFEE33FEED33FDCC33CCC833C810D7079C
:102A83009BEC9AE899400AED9BFDEC9AFCE899F8D7
:0E2A93000FD5F0DAE4CDFBE4CCFAE4C8F9226A
:0E2AA100C3E49FFFE49EFEE49DFDE49CFC2246
:102AAF00EB9FF5F0EA9E42F0E99D42F0E89C45F07D
:012ABF0022F4
:0C2AC000ECF0A3EDF0A3EEF0A3EFF02289
:102ACC00A8828583F0D083D082122AE3122AE312E3
:102ADC002AE3122AE3E473E493A3C583C5F0C58308
:102AEC00C8C582C8F0A3C583C5F0C583C8C582C854
:012AFC0022B7
:1022D200E53B242FF8E6053B22782C302702782FA5
:1022E200E475F001122B5E0229382020EB7F2ED2FA
:1022F200208018EF540F2490D43440D4FF30240BA4
:10230200EF24BFB41A0050032461FFE53C600215BC
:102312003C053FE53F7002053E30270D782CE47501
:10232200F001122B5EEF022AFD024CF77403D22752
:102332008003E4C227F53B8B2C8A2D892EE4F53CE1
:10234200F53EF53FE53C60077F2012230D80F575D1
:102352003DFFC221C220C222C223C225C226C228F8
:102362001222DBFF700D3027057F0012231EAF3FC4
:10237200AE3E22B4255FC2D5C2241222DBFF24D096
:10238200B40A00501A75F00A783C30D50508B6FF39
:102392000106C6A426F620D5047002D22380D924D1
:1023A200CFB41A00EF5004C2E5D22402251ED22176
:1023B20080C6D22080C0D22280BCD2D580BAD2259B
:1023C20080B47F2012230D2022077401B53C004007
:1023D200F11222D2FF12230D022346D228D22680E6
:1023E200951222D2FB1222D2FA1222D2F94A4B7051
:1023F2000679EF7A257BFF20222EE53C602A7E00BB
:102402008E8275830012295160060EEE653D70F0D2
:10241200C2D5EBC0E0EAC0E0E9C0E0EE122565D02B
:10242200E0F9D0E0FAD0E0FB122938FF60AAEBC055
:10243200E0EAC0E0E9C0E012230DD0E02401F9D0C7
:10244200E03400FAD0E0FBE53D0460DCD53DD98004
:10245200877BFF7A257961D222809C79108002796C
:1024620008C226C2288008D2D5790A8004790AC215
:10247200D5E53D047002F53DE4FAFDFEFF1222D2DD
:10248200FC7B082021131222D2FD7B1030200A127D
:1024920022D2FE1222D2FF7B20EC3382D592D5507B
:1024A20013C3E43020069FFFE49EFEE42021039D37
:1024B200FDE49CFCE4CBF8C221EC700CCFCECDCC79
:1024C200E824F8F870F38017C3EF33FFEE33FEED24
:1024D20033FDEC33FCEB33FB994002FB0FD8E9EB05
:1024E200302105F8D0E0C448B221C0E00AEC4D4EDC
:1024F2004F78207B0070C2EAB53D0040BCC0E012BC
:102502002567D0F0D0E0202104C4C0E0C4B221C0CD
:10251200F01222F6D0F0D5F0EB022346122BBD23A7
:10252200E353245D5823B44C23B04224614F246901
:0F2532004424694923C943246F55245346245335
:1025410045245347260F5023B82D23BC2E23DF2BC0
:1025510023C02323DD2025F82A237848000023D730
:102561003F3F3F00790AA2D5202314302509B91035
:10257100020404B9080104A2D52026025001042056
:1025810022689222B53C005034C0E07F20302319EC
:102591007F30A22272267225500F1225BEC222C29E
:1025A10026C225C2287F30800F302503E9C0E01202
:1025B100230D302503D0E0F9D0E0B53CCC30251710
:1025C1007F30B9100C12230D7F583024077F78809B
:1025D10003B9080312230D3022057F2D02230D7F3D
:1025E100202028F87F2B2026F322922280CF286EEC
:1025F100756C6C2900D2211222D23021F8C22178C7
:102601003C30D50108F60223782D50434958122257
:10261100D22403B405004001E490260A931222FE5D
:0D262100743A1222FED223753C0402245D9F
:10343B008B2F8A308931E4F53BF53AF539F538F5C0
:10344B0036F537E533453445326012EBC0E0EAC060
:10345B00E0E9C0E0AB32AA33A934122B6EAB2F05D7
:10346B0031E531AA307002053014F9122938F53CD8
:10347B00C394094007E53CD3940D40E1E53C64203F
:10348B0060DBE53CB42D054337038016E53CB42BDC
:10349B0005433701800C74FF2531F53174FF35304E
:1034AB00F530E53560046410703FAB2FAA30A931BD
:1034BB0012293864306009E535702E75350A80297C
:1034CB00900001122951FF64786004EFB458134344
:1034DB00370175351074022531F531E43530F5308F
:1034EB008007E5357003753508AB2F0531E531AA3B
:1034FB00307002053014F9122938F53CC394614041
:10350B000AE53CD3947A5003533CDF74D0253CF549
:10351B003CC3940A400CE53C9411406D74F9253C76
:10352B00F53CE53CD395355060433701853B4085F1
:10353B003A3F85393E85383DAF357E00E4FCFDAB27
:10354B003BAA3AA939A838122B0FC8ECC8C9EDC948
:10355B00CAEECACBEFCBE4FCFDFEEB253CF53BEE14
:10356B003AF53AED39F539EC38F538AF3BAE3AADC3
:10357B0039FCAB40AA3FA93EA83DD3122AAF50035A
:10358B000234F44337040234F4E53720E003E480DB
:10359B002DE53345344532601EAB2FE53124FFF961
:1035AB00E53034FFFAEBC0E0EAC0E0E9C0E0AB3253
:1035BB00AA33A934122B6EE53730E20774FFFFFEF6
:1035CB00FDFC22E537AF3BAE3AAD39AC3830E10309
:0435DB00022AA122FD
:102AFD00BB010689828A83F0225002F722BBFE01B8
:022B0D00F322B1
:102B0F00E88FF0A4CC8BF0A42CFCE98EF0A42CFC65
:102B1F008AF0EDA42CFCEA8EF0A4CDA8F08BF0A4E3
:102B2F002DCC3825F0FDE98FF0A42CCD35F0FCEB42
:102B3F008EF0A4FEA9F0EB8FF0A4CFC5F02ECD3907
:0F2B4F00FEE43CFCEAA42DCE35F0FDE43CFC2274
:102B5E00FAE6FB0808E6F925F0F618E6CA3AF62278
:102B6E00BB011A89828A83D0F0D0E0F8D0E0F9D088
:102B7E00E0FAD0E0FBE8C0E0C0F0022BEC5016E922
:102B8E00F8D083D082D0E0F9D0E0FAD0E0FBC0825A
:102B9E00C083022BE3BBFE16E9F8D083D082D0E0CF
:0F2BAE00F9D0E0FAD0E0FBC082C083022BF52201
:102BBD00D083D082F8E4937012740193700DA3A3A7
:102BCD0093F8740193F5828883E4737402936860BB
:062BDD00EFA3A3A380DFBB
:092BE300EBF608EAF608E9F62217
:092BEC00EBF0A3EAF0A3E9F022EA
:092BF500EBF208EAF208E9F22211
:00000001FF
